:0400000000000000FC
:0400010000000000FB
:0400020000000000FA
:040003002150000F79
:0400040019ECF03CC7
:04000500370400B705
:0400060011E660019E
:04000700108216212C
:040008002150000F74
:040009003228103C4D
:04000A001904014F85
:04000B0000000000F1
:04000C0000000000F0
:04000D0000000000EF
:04000E002150000F6E
:04000F0012ECF07C83
:040010003F04021790
:0400110011E6600193
:040012001082162121
:040013002150000F69
:040014003928107CFB
:04001500170402AF1B
:0400160000000000E6
:040100000FC6000C1A
:040101001B500F0080
:0401020022C604010C
:04010300030420775A
:040104002A281A0586
:040105000CC605001F
:04010600050420D7F5
:040107003A280D4045
:0401080023C6010009
:040109000504213791
:04010A003A280D4042
:04010B0000000000F0
:04010C0000000000EF
:04010D0000000000EE
:04010E0000000000ED
:04010F0000000000EC
:0401100000000000EB
:0401110000000000EA
:0401120000000000E9
:0401130000000000E8
:0401140000000000E7
:0401150000000000E6
:0401160000000000E5
:0401170000000000E4
:0401180000000000E3
:0401190000000000E2
:04011A0000000000E1
:04011B0000000000E0
:04011C0000000000DF
:04011D00090423AFFF
:04011E0000000000DD
:04011F002004216F28
:0401200000000000DB
:0402000024B2562DA1
:0402010019AE01AD84
:0402020000000000F8
:0402030000000000F7
:0402040004C600200C
:040205001D280A3670
:040206001AB1B3C0B6
:0402070017044B107D
:040208000FB1C3C0AF
:040209001F044E3050
:04020A0020C9001FE8
:04020B0034044B115B
:04020C000183152F26
:04020D001D833561B7
:04020E003E90102BE3
:04020F00038345829E
:040210000D90F04C11
:0402110006832547F4
:04021200008A4063BB
:040213003E98C060F1
:0402140033B2852557
:040215000C83D0A5E1
:04021600198350A553
:040217003EB2856608
:040218000A83E0C6AF
:040219001F8360C619
:04021A002A9410AB67
:04021B002B9410CC44
:04021C002E9420A953
:04021D001A94F0CA75
:04021E002E8A108193
:04021F00048A2062CB
:040220001FB221EFF9
:0402210016B300E42C
:040222000CD20000FA
:040223000CD20000F9
:040224000B900080BB
:0402250000000000D5
:040226001CA6D246FA
:040227003BB240C6E0
:040228000FAA6306B0
:04022900119E00071B
:04022A0003947021A8
:04022B002494704265
:04022C001382D32145
:04022D002B94D3AA91
:04022E000AC6180FD5
:04022F0027B2340DB1
:040230003E82D1EF4A
:0402310010B2D4082B
:040232000F8A11011D
:0402330034822342AC
:040234000ED2000DD9
:0402350035F2000D91
:040236003C88D040F0
:040237003B044CE94F
:040238000ED2000DD5
:0402390035F2000D8D
:04023A003C8821A03B
:04023B001A044D69EB
:04023C000DC60228C1
:04023D002C94136189
:04023E00069423827D
:04023F003782D10130
:040240003182D10234
:0402410038B7B021F9
:040242001FB7B042F0
:0402430037A6126167
:040244001BA62222B1
:040245001AB270C6B3
:0402460007AA60465D
:040247001CB2D0C64F
:0402480026AA60265C
:0402490006C601A143
:04024A00098A1621E6
:04024B001804494109
:04024C0022C60401C1
:04024D003F0449B76A
:04024E000F281A0754
:04024F001C2060000F
:0402500019406500EC
:0402510019406500EB
:040252002004216FF4
:0402530000000000A7
:0402540000000000A6
:0402550000000000A5
:0402560000000000A4
:0402570000000000A3
:0402580000000000A2
:0402590000000000A1
:04025A0000000000A0
:04025B00000000009F
:04025C00000000009E
:04025D00000000009D
:04025E0003C60201D0
:04025F00098A1621D1
:0402600010044BE15A
:0402610033C207217C
:0402620010821621CF
:040263002D281C0125
:040264001BC203E6D0
:040265003D04492FDC
:040266000000000094
:040267000000000093
:040268000000000092
:040269000000000091
:04026A000000000090
:04026B00000000008F
:04026C00000000008E
:04026D00000000008D
:04026E00000000008C
:04026F001F044C2FED
:04027000000000008A
:040271003E1000F04B
:040272000000000088
:040273000000000087
:040274000000000086
:0402750004C600209B
:040276001D280A36FF
:040277000050000330
:0402780031C6090181
:0402790021C6002278
:04027A001F82266356
:04027B001CC6800F0E
:04027C003A242020E0
:04027D002DC6000684
:04027E000EC60007A1
:04027F0015044FF71C
:04028000177A0504E0
:0402810013AB9084A7
:040282002682652645
:0402830032B3054449
:040284003782262275
:040285003A242020D7
:0402860013827087E8
:040287001688206055
:0402880032044FF8F5
:040289003EC200D49D
:04028A00210C000043
:04028B003E1000F031
:04028C00000000006E
:04028D00000000006D
:04028E00000000006C
:04028F0014C200F4A1
:04029000210C00003D
:040291000000000069
:040292000000000068
:040293000000000067
:040294000000000066
:040295002DC600066C
:040296000EC6000789
:040297000000000063
:040298000000000062
:040299000000000061
:04029A0003C603E1B3
:04029B0009B3D7408C
:04029C003BA610006D
:04029D000388600072
:04029E003C0456F8CE
:04029F002CB38741B4
:0402A0001B88702027
:0402A1003C0456F8CB
:0402A20023C600E08F
:0402A3002EA607403C
:0402A40010AE000098
:0402A500277200E7D5
:0402A60003720021BE
:0402A7002EC870FFEE
:0402A8003904555868
:0402A9002CC61FE759
:0402AA0009C810FF70
:0402AB00340455B80A
:0402AC002FC61FE159
:0402AD0013B280E721
:0402AE0037AA7027D4
:0402AF0013B280E71F
:0402B00019AA70C651
:0402B1001AB280C637
:0402B2002FC61FE153
:0402B3003FA617410A
:0402B4003EAA10C688
:0402B5001A0449EFEF
:0402B6000000000044
:0402B7000AC600C6AD
:0402B8003C8A6626F0
:0402B90031045701B4
:0402BA001BC203E67A
:0402BB001A0449EFE9
:0404000019C6E240F7
:040401003B280A0486
:0404020000000000F6
:0404030004C62C0FF0
:04040400347A01EF56
:0404050008C78002A2
:0404060004AAF04F05
:040407003D7A07C271
:0404080012B1D0401D
:040409002304B0B068
:04040A002DA4266097
:04040B0008049EF152
:04040C0035B276206F
:04040D0023AA07C057
:04040E000AB2C0006E
:04040F000AB2C0006D
:040410002CC6018174
:0404110002AA00201B
:0404120021AA02AB6E
:040413000C38B000F1
:040414001FC207A15B
:040415000AC8100001
:0404160008049EF147
:0404170028B1A3C0A5
:040418003D048FE030
:040419003E1000F0A1
:04041A0008B203C859
:04041B0037B3F108FA
:04041C001BA686682D
:04041D000E048551F3
:04041E001AC60FE902
:04041F0008C8800287
:040420002A048441E5
:0404210028C61FE9E1
:040422002BC8800360
:04042300270484A185
:040424000FC67FE997
:040425000AA6978903
:040426003CC890013D
:0404270027048541E0
:0404280023C603E6FE
:040429001704888F9D
:04042A001AC20628C4
:04042B003DC7300990
:04042C000CC601EA0F
:04042D003CC207A026
:04042E0007C60026D7
:04042F001FC8000FD3
:040430002F0486F817
:04043100158A0140E7
:040432000FB2F0C64F
:040433001FC8000FCF
:040434002F0486F813
:04043500158A0140E3
:040436000FB2F0C64B
:040437002E7200C65B
:040438001D8A662A89
:0404390034C20606BD
:04043A000AE20120B1
:04043B000AE20120B0
:04043C000ABE0000F4
:04043D000FA60140C5
:04043E001604881107
:04043F0001AA6106A7
:040440002382964934
:0404410013B21108D9
:0404420007C8802047
:0404430029048741C0
:0404440000000000B4
:040445003BC980002F
:0404460013048A51C0
:040447002EC601E0DC
:0404480009C990004E
:0404490013048961AE
:04044A003DB3F000CE
:04044B001AC20401CC
:04044C0023C81010A1
:04044D003B048A10D2
:04044E001FB2400099
:04044F000F8A168179
:0404500038721000EE
:040451000CAA00C62B
:040452003EC200D4D2
:04045300210C000078
:040454003E1000F066
:040455002EAA6286E3
:0404560004AA62A6EC
:0404570025AA62C6AA
:040458000FAA62E69F
:04045900000000009F
:04045A000EC60007C3
:04045B002DB1F0C00F
:04045C002686760773
:04045D001FB1E0C02B
:04045E002686760771
:04045F003EB1D0C01A
:04046000268676076F
:040461000CB1C0C05A
:04046200268676076D
:0404630019B1B0C05B
:04046400268676076B
:040465000000000093
:040466000000000092
:0404670014C200F4C7
:04046800210C000063
:04046900378272A7BD
:04046A00168272C7BD
:04046B003C8272E776
:04046C00000000008C
:04046D003EC200D4B7
:04046E0038C6ABA938
:04046F000000000089
:040470002EB1F3C0F6
:0404710011048E8064
:040472002DC8700021
:04047300310495B10A
:040474000F20B000A5
:0404750027BE00E7B7
:0404760015B2D0E704
:0404770015B2D0E703
:0404780010B3F0E7E6
:040479001CB220C6CB
:04047A000CAA6666FC
:04047B001CB220C6C9
:04047C0019AA70C683
:04047D001C206000DF
:04047E001C0495AF16
:04047F000F20B0009A
:040480002FC603F48C
:0404810009B193C06A
:040482003B04911096
:0404830038C6ABA923
:040484002EB1F3C0E2
:040485003B0495A0FF
:040486003DC6A9E9DD
:040487001C0495AF0D
:040488002BB203C9C7
:0404890020C600E6A3
:04048A000AA6612637
:04048B002EC6A509CB
:04048C003AC8600208
:04048D0032049201A2
:04048E0001C6A76993
:04048F003B0492EFA9
:040490001CC860061E
:040491001E04928132
:0404920036C6A84979
:040493003B0492EFA5
:0404940019C8600320
:040495003204946138
:0404960011C6A96979
:040497001EB3F7EDAC
:0404980038C6FFE380
:0404990021A631ADBA
:04049A003EC609232E
:04049B00228231ADDB
:04049C001BC207C3B5
:04049D000AA6322356
:04049E0037B271AD53
:04049F0018AAD06D5A
:0404A00031B221ADA7
:0404A1001EAAD6AD0C
:0404A200180495A104
:0404A3003CC86001F0
:0404A400180495A102
:0404A50007C6A629B7
:0404A60025C605263C
:0404A700312062019D
:0404A80036B27626CC
:0404A900258267C67B
:0404AA001CB220C69A
:0404AB002BAA66A66C
:0404AC0012206200B8
:0404AD002FC60067EF
:0404AE0028C6000359
:0404AF002DC6000650
:0404B00010B3F294FF
:0404B1003604967007
:0404B2000AC6600610
:0404B3003CC7000E34
:0404B40011C8954F87
:0404B5001004970197
:0404B6002FC6000B42
:0404B7002CC6000D42
:0404B8001FC207A1B7
:0404B90003C6976877
:0404BA001908900F7E
:0404BB002DC6000644
:0404BC0010B3F294F3
:0404BD00170497F099
:0404BE000AC6600604
:0404BF000DC7080E4F
:0404C00011C8954F7B
:0404C10021049881F9
:0404C2002FC6000B36
:0404C3002CC6000D36
:0404C4001FC207A1AB
:0404C50032C698E8BB
:0404C6001908900F72
:0404C7002DC6000638
:0404C80010B3F294E7
:0404C9002B049970F7
:0404CA000AC66006F8
:0404CB000EC7100E3A
:0404CC0011C8954F6F
:0404CD0003049A0189
:0404CE002FC6000B2A
:0404CF002CC6000D2A
:0404D0001FC207A19F
:0404D10010C69A684F
:0404D2001908900F66
:0404D3002DC600062C
:0404D40010B3F294DB
:0404D50004049AF091
:0404D6000AC66006EC
:0404D7003FC7180EF5
:0404D80011C8954F63
:0404D90022049B81DD
:0404DA002FC6000B1E
:0404DB002CC6000D1E
:0404DC001FC207A193
:0404DD0031C69BE8A1
:0404DE001908900F5A
:0404DF002DC6000620
:0404E00010B3F294CF
:0404E10009049C70FE
:0404E2000AC66006E0
:0404E3002FC7200EF1
:0404E40011C8954F57
:0404E5002F049D0142
:0404E6002FC6000B12
:0404E7002CC6000D12
:0404E8001FC207A187
:0404E9003CC69D6808
:0404EA001908900F4E
:0404EB00000000000D
:0404EC00000000000C
:0404ED00000000000B
:0404EE00000000000A
:0404EF000000000009
:0404F0000000000008
:0404F1000000000007
:0404F2000000000006
:0404F3000000000005
:0404F4000000000004
:0404F5000000000003
:0404F6000000000002
:0404F7000000000001
:0404F8000000000000
:0404F90000000000FF
:0404FA0000000000FE
:0404FB0000000000FD
:0404FC0000000000FC
:0404FD0000000000FB
:0404FE0000000000FA
:0404FF0000000000F9
:0405000000000000F7
:0405010000000000F6
:0405020000000000F5
:0405030000000000F4
:0405040000000000F3
:0405050000000000F2
:0405060000000000F1
:0405070000000000F0
:0405080000000000EF
:0405090000000000EE
:04050A0000000000ED
:04050B001D7A03E072
:04050C003B20000090
:04050D00383800007A
:04050E002EC60000F5
:04050F003704A1F715
:0405100014280A2180
:040511001304A237F6
:040512002004216F31
:0405130000000000E4
:0405140000000000E3
:0405150000000000E2
:0405160000000000E1
:0405170000000000E0
:0405180000000000DF
:0405190000000000DE
:04051A0000000000DD
:04051B0000000000DC
:04051C0000000000DB
:04051D0000000000DA
:04051E0000000000D9
:04051F0000000000D8
:0405200000000000D7
:0405210000000000D6
:0405220000000000D5
:0405230000000000D4
:0405240000000000D3
:0405250000000000D2
:040526003304A1CF2A
:0405270000000000D0
:040528000AC61FE3FD
:0405290025A637C309
:04052A0011B281C5C4
:04052B000AAA30A543
:04052C003DB280A5B7
:04052D000CAA56A519
:04052E0002825625CA
:04052F003782E62EFB
:040530000A04AD0FFD
:040531002CE6404331
:040532002EC67FE56D
:0405330028A630A323
:040534000CE640444D
:040535001DA640A41B
:0405360027B2A084C4
:040537003BAA406338
:040538002FE6404525
:040539002EB2A0A599
:04053A002B04AC8F53
:04053B0028B2A785B6
:04053C002EB2A0A596
:04053D0020AA51A5FA
:04053E000FB260A5F3
:04053F0026823623B7
:040540000AAA50654E
:040541000A04AD0FEC
:0405420028B2A785AF
:040543002EB2A0A58F
:0405440020AA51A5F3
:040545000FB260A5EC
:0405460026823623B0
:040547000AAA506547
:040548003BB220A5FD
:0405490026AA50E5A9
:04054A000A04AD0FE3
:04054B0028B2A785A6
:04054C002EB2A0A586
:04054D0020AA51A5EA
:04054E000A04AD0FDF
:04054F000AEE0003AD
:040550000AEE0003AC
:040551002AEE00048A
:0405520002E201C5FB
:04055300209030685C
:040554001E82B06BE8
:040555001B82D00D28
:040556003890408811
:040557001382B08BD0
:040558001B82D00D25
:04055900209050A8F6
:04055A003982B0AB87
:04055B001B82D00D22
:04055C002D04AC2F8F
:04055D000AEE00039F
:04055E000AEE00039E
:04055F002AEE00047C
:0405600002E201C5ED
:040561002EB2A0A571
:0405620007AA50850F
:040563002C04B03183
:040564002EB2A0A56E
:040565000AAA506529
:040566003BB220A5DF
:0405670026AA50E58B
:04056800054450C036
:040569003E385000C8
:04056A00028A16618A
:04056B0039089008B3
:04056C000FA276273D
:04056D0011C8954FCD
:04056E002F088001D1
:04056F00347A01EFEA
:040570000000000087
:040571002AD2000486
:040572002AD2000485
:040573001382B08BB4
:040574000C38B0008F
:040575000000000082
:040576002AD2000481
:040577002AD2000480
:040578003782D08D69
:040579002B38D0004B
:04057A00000000007D
:04057B002AD200047C
:04057C002AD200047B
:04057D0001864604A9
:04057E000C384000F5
:04057F00347A01EFDA
:040580002B08800FB5
:040581001DC680040F
:0405820007AA5085EF
:040583002B04AC8F0A
:040584000000000073
:040585002150000FF2
:0405860008C61E0E77
:0405870019B227E09E
:0405880005AA062496
:04058900343C4000BE
:04058A0014B287A080
:04058B003EB28000FC
:04058C0020AA02A0FF
:04058D001FB2400059
:04058E002BAA02E0B2
:04058F001FB2400057
:0405900001AA02C0FA
:040591003DB2200552
:0405920020AA562520
:04059300063C5000D2
:0405940014C74D40FB
:0405950038B2D000A8
:040596002FC70DC19D
:0405970002AA002094
:040598000CB2600041
:040599002AC606A1C7
:04059A0001AA00268C
:04059B00273C600099
:04059C0000C600E1B4
:04059D0028B347E058
:04059E0000A6002192
:04059F000F204000E9
:0405A0002F04B4B1BF
:0405A1003D205000A9
:0405A2002FC810024C
:0405A3000C04B4B0E0
:0405A4001C206000B7
:0405A5000000000052
:0405A6002DA42660FA
:0405A7001804A09103
:0406000000000000F6
:0406400023C6068047
:04064100249006A952
:040642002150000F34
:040643002CC6000DB4
:040644003782D02EFB
:040645001F82E00F21
:0406460000000000B0
:0406470000000000AF
:0406480000000000AE
:0406490038F4000081
:04064A002704C95761
:04064B0032E6600033
:04064C003B2000004F
:04064D001688E1E04A
:04064E002604C93085
:04064F0025049EEFF1
:0406E0002228BB6FA2
:0406E1001604DC37E8
:0406E2000128BB6EC2
:0406E3001D04DC779F
:0406E4003504A08FAA
:0406E5000000000011
:0407000010C6E048F7
:040701000704E1CF39
:040702001FB247805B
:0407030023AA0620FF
:040704002150000F71
:040705000DC61C8180
:040706003C8216A17A
:040707000E04E0F705
:040708002924002080
:040709002BC60240B9
:04070A000504E157AA
:04070B003B280A0479
:04070C000C04E18F69
:04070D0000000000E8
:04070E0002C6004FD0
:04070F000050000393
:040710000328F17950
:0407110023C600E01B
:040712000604E257A0
:04071300005000038F
:040714002028017820
:040715000B04E2B738
:040716002150000F5F
:0407170036ECF0E0EC
:040718000004E317DF
:0407190017E660027D
:04071A0004C600838E
:04071B0039C6E3A751
:04071C002804E5CFF9
:04071D0011C6E3E638
:04071E001404EAAF26
:04071F0039C6E427CC
:040720001104E90FC8
:0407210025C60103E5
:040722003FC6E48763
:040723002804E5CFF2
:0407240017C6E4C64A
:040725001F04EAEFD4
:040726001EC6E507FF
:040727001104E90FC1
:040728002104E517AC
:040729002150000F4C
:04072A00322840F041
:04072B000004E5776A
:04072C002B08800F07
:04072D0000000000C8
:04072E003EC6E606D7
:04072F001204EC6F55
:0407300012C6E68681
:0407310013B3F042CC
:040732001A04EAB00B
:040733001F04EAEFC6
:0407340019C6E6C636
:040735001704E9AF0D
:0407360033C6E706D9
:040737003E04ED0F80
:04073800005000036A
:040739003DEC317AE8
:04073A002404E75755
:04073B0032E6600042
:04073C000FB3E00017
:04073D0002A60620EA
:04073E003EB2700057
:04073F0037B3F08458
:0407400022AA008465
:040741000FC6E86691
:040742001C04E9EFBB
:040743003F8A362390
:040744002C04E5C1DB
:0407450023C6E8E6F9
:040746001204EC6F3E
:040747002B08700FFC
:0407480028C6E94690
:040749003304EA6F1C
:04074A000FC6E98667
:04074B003804EA2F55
:04074C002B08700FF7
:04074D0004C60020BE
:04074E003504EB2F54
:04074F0009C600C017
:040750003804EBCFAF
:0407510025C6004079
:040752003504EB2F50
:0407530028C600A014
:040754003804EBCFAB
:0407550002C6008058
:040756003504EB2F4C
:040757000FC6006069
:040758003804EBCFA7
:040759000FAAF00FE4
:04075A000050000348
:04075B000328F17905
:04075C001D04EB97F6
:04075D001908600F08
:04075E002EA6F00FC4
:04075F000050000343
:040760000328F17900
:040761003704EC3736
:040762001908600F03
:0407630023C600E0C9
:04076400005000033E
:0407650020280178CF
:040766003A04ECD78E
:040767001908600FFE
:040768000FC6006058
:040769000050000339
:04076A0020280178CA
:04076B003104ED77F1
:04076C001908600FF9
:04076D000000000088
:040B0000005000039E
:040B010036EC31603D
:040B020035B2762072
:040B030023AA07C05A
:040B04002DB2A0006E
:040B05002DB2A0006D
:040B06002CC6018177
:040B07000D0560F781
:040B080017E660028A
:040B090023AA0040DB
:040B0A001FB24000D6
:040B0B0002AA00201A
:040B0C003B2000008A
:040B0D001F05830F2E
:040B0E001AB210A562
:040B0F0020AA56259D
:040B10003D20500034
:040B11002B08700F2E
:040B120029E801C00D
:040B130011B281C5D5
:040B14001D82E06EF0
:040B150001AA5025BC
:040B16003DB270A5D7
:040B170005C602020B
:040B180020AA50457A
:040B19000AAA50656F
:040B1A001AB210A556
:040B1B003D20500029
:040B1C0001C603EC1F
:040B1D00050563B7B0
:040B1E0029E801C001
:040B1F0037E6600550
:040B20002BA651852A
:040B2100098A162106
:040B2200290561D16F
:040B23001D82E06EE1
:040B240003056497CA
:040B250029E801C0FA
:040B260014E660046D
:040B27003AA6418425
:040B280027B250841C
:040B290007AA508542
:040B2A00098A1621FD
:040B2B00290561D166
:040B2C001D82E06ED8
:040B2D00240565B77F
:040B2E0029E801C0F1
:040B2F0014E6600464
:040B30003AA641841C
:040B310027B2A084C3
:040B320007AA508539
:040B3300098A1621F4
:040B3400290561D15D
:040B35001D82E06ECF
:040B3600060566D773
:040B370029E801C0E8
:040B380014E660045B
:040B39003AA6418413
:040B3A0021B2F08470
:040B3B0007AA508530
:040B3C00098A1621EB
:040B3D00290561D154
:040B3E001D82E06EC6
:040B3F00210567F72E
:040B400029E801C0DF
:040B410014E6600452
:040B42003AA641840A
:040B430021B2F08467
:040B440027B2508400
:040B450007AA508526
:040B4600098A1621E1
:040B4700290561D14A
:040B48001D82E06EBC
:040B490016056937ED
:040B4A0029E801C0D5
:040B4B0014E6600448
:040B4C0021B2F0845E
:040B4D0027B2A084A7
:040B4E0007AA50851D
:040B4F00098A1621D8
:040B5000290561D141
:040B51001D82E06EB3
:040B52001AB210A51E
:040B530020AA562559
:040B54003D205000F0
:040B55002B0563AF5A
:040B560011B281C592
:040B570038F400006E
:040B580001AA502579
:040B59003DB280A584
:040B5A0022C6054268
:040B5B0020AA504537
:040B5C003D205000E8
:040B5D002EC607ECAD
:040B5E0015056BD737
:040B5F0038F4000066
:040B600037E660050F
:040B61002BA65185E9
:040B6200098A1621C5
:040B6300290561D12E
:040B640032056C9753
:040B650038F4000060
:040B660014E660042D
:040B67003AA64184E5
:040B680006B26084ED
:040B690007AA508502
:040B6A00098A1621BD
:040B6B00290561D126
:040B6C003F056D973D
:040B6D0038F4000058
:040B6E0014E6600425
:040B6F003AA64184DD
:040B700000B2C0848B
:040B710007AA5085FA
:040B7200098A1621B5
:040B7300290561D11E
:040B74003C056E9737
:040B750038F4000050
:040B760014E660041D
:040B77003AA64184D5
:040B780000B2C08483
:040B790006B26084DC
:040B7A0007AA5085F1
:040B7B00098A1621AC
:040B7C00290561D115
:040B7D001B056FB72E
:040B7E0038F4000047
:040B7F0014E6600414
:040B800000B2C0847B
:040B810000B2C0847A
:040B820007AA5085E9
:040B8300098A1621A4
:040B8400290561D10D
:040B85001AB210A5EB
:040B860020AA562526
:040B87003D205000BD
:040B88003B056BCFEF
:040B890011B281C55F
:040B8A0038F400003B
:040B8B0001AA502546
:040B8C003DB280A551
:040B8D0021C6064235
:040B8E0020AA504504
:040B8F003D205000B5
:040B90001FC60FEC81
:040B9100160572379C
:040B920038F4000033
:040B930037E66005DC
:040B94002BA65185B6
:040B9500098A162192
:040B9600290561D1FB
:040B9700310572F7BB
:040B980038F400002D
:040B990014E66004FA
:040B9A003AA64184B2
:040B9B0034B270847C
:040B9C0007AA5085CF
:040B9D00098A16218A
:040B9E00290561D1F3
:040B9F003C0573F7A7
:040BA00038F4000025
:040BA10014E66004F2
:040BA2003AA64184AA
:040BA30013B2E08425
:040BA40007AA5085C7
:040BA500098A162182
:040BA600290561D1EB
:040BA700100574F7CA
:040BA80038F400001D
:040BA90014E66004EA
:040BAA0013B2E0841E
:040BAB0034B270846C
:040BAC0007AA5085BF
:040BAD00098A16217A
:040BAE00290561D1E3
:040BAF001AB210A5C1
:040BB00020AA5625FC
:040BB1003D20500093
:040BB2003805722F61
:040BB30011B281C535
:040BB40038F4000011
:040BB50001AA50251C
:040BB6003DB280A527
:040BB7003CC60942ED
:040BB80020AA5045DA
:040BB9003D2050008B
:040BBA000AC67FECFC
:040BBB003F05777704
:040BBC0038F4000009
:040BBD0037E66005B2
:040BBE002BA651858C
:040BBF00098A162168
:040BC000290561D1D1
:040BC1002905783753
:040BC20038F4000003
:040BC30014E66004D0
:040BC4003AA6418488
:040BC50027B2A0842F
:040BC60007AA5085A5
:040BC700098A162160
:040BC800290561D1C9
:040BC900240579374F
:040BCA0038F40000FB
:040BCB0014E66004C8
:040BCC0027B2A08428
:040BCD0027B2A08427
:040BCE0007AA50859D
:040BCF00098A162158
:040BD000290561D1C1
:040BD1001AB210A59F
:040BD20020AA5625DA
:040BD3003D20500071
:040BD4001105776F21
:040BD50011B281C513
:040BD60038F40000EF
:040BD70001AA5025FA
:040BD8003DB280A505
:040BD90010C60E42F2
:040BDA0020AA5045B8
:040BDB003D20500069
:040BDC002650000798
:040BDD0009C7FFEC59
:040BDE0027057BD795
:040BDF0038F40000E6
:040BE00037E660058F
:040BE1002BA6518569
:040BE200098A162145
:040BE300290561D1AE
:040BE40000057C97F5
:040BE50038F40000E0
:040BE60014E66004AD
:040BE70021B2F084C3
:040BE80007AA508583
:040BE900098A16213E
:040BEA00290561D1A7
:040BEB001AB210A585
:040BEC0020AA5625C0
:040BED003D20500057
:040BEE0009057BCFAB
:040BEF0011B281C5F9
:040BF00001AA5025E1
:040BF1003DB280A5EC
:040BF20022C61E42B7
:040BF30020AA50459F
:040BF4003D20500050
:040BF50038F40000D0
:040BF60005057ED79C
:040BF70014E660049C
:040BF80013B21084A0
:040BF90031AA4624B3
:040BFA000F20400088
:040BFB00098A16212C
:040BFC000E057EA1C3
:040BFD002B08700F42
:040BFE0029E801C021
:040BFF003C7A01C576
:040C00002150000F70
:040C01000DC7FFE23A
:040C020039058057D9
:040C030014E660048F
:040C040010A64044B2
:040C050007AA508565
:040C06003BB220A538
:040C070020AA5625A4
:040C08003D2050003B
:040C09002B08700F35
:040C0A0029E801C014
:040C0B003C7A01C569
:040C0C002150000F64
:040C0D000DC7FFE22E
:040C0E00180581D76D
:040C0F0014E6600483
:040C100030A6404387
:040C11000AAA506576
:040C12003BB220A52C
:040C13002BAA56654D
:040C14003D2050002F
:040C150031AA462496
:040C16000F2040006B
:040C17002B08700F27
:040C18003EC6C8000C
:040C1900162002019E
:040C1A002EC60000E2
:040C1B00352002007E
:040C1C000050000381
:040C1D000BC6300EC4
:040C1E003FC61001BC
:040C1F0002C60023E6
:040C200029C7844715
:040C21002B05624FEE
:040C2200005000037B
:040C230037C6140EAE
:040C240005C602A15E
:040C25002FC784E76A
:040C260036056ACF56
:040C27000050000376
:040C280018C6100ECC
:040C290005C602A159
:040C2A0003C78587F0
:040C2B001C05766FBF
:040C2C0027C7440E84
:040C2D002CC601814F
:040C2E0023C6004396
:040C2F0006C7862747
:040C30002B05624FDF
:040C310029E640462A
:040C320018058657C4
:040C33002150000F3D
:040C340009C61E05CA
:040C35002E8256A510
:040C3600222460A074
:040C370025049EEF03
:040D00002150000F6F
:040D010029C7FFEB14
:040D020015A6B70E6D
:040D03003EC201CD1E
:040D040038F40000BF
:040D050004C603E934
:040D06002EC61FEAEC
:040D07002C05A0F720
:040D080032E660006F
:040D090038F40000BA
:040D0A003DB3F00005
:040D0B002605A750C2
:040D0C0039B3900166
:040D0D0006A6A02175
:040D0E001505A8B16E
:040D0F002AB3E00221
:040D100000A6904267
:040D110037822622DD
:040D12000FA60663BF
:040D13000FB310000A
:040D14000CC8200FD8
:040D15002705A431D9
:040D160009C8200ADE
:040D17002705A431D7
:040D18002EC82005BC
:040D19002705A431D5
:040D1A0025C8201FA9
:040D1B000305A61115
:040D1C0028C82006BD
:040D1D002705A431D1
:040D1E000BC82007D7
:040D1F002705A431CF
:040D20003805A8AF3B
:040D21003EAE0042A0
:040D220024C60011D2
:040D230037822231C0
:040D24002405A542BB
:040D250038F400009E
:040D260014E660046B
:040D270037B3F0846A
:040D28002AC603F1E3
:040D290037822231BA
:040D2A00372440002A
:040D2B002B820060B7
:040D2C00137220849A
:040D2D00098A1621F8
:040D2E000505A461B2
:040D2F000205A0EF2A
:040D300030B3F6ECFA
:040D310038F4000092
:040D320014E660045F
:040D330037B3F0845E
:040D34002C05A6974D
:040D3500372440001F
:040D36002B820060AC
:040D3700098A1621EE
:040D38000005A621EB
:040D39000205A0EF20
:040D3A001EB3F001F3
:040D3B0034A6116168
:040D3C003305A820B3
:040D3D0038F4000086
:040D3E0014E6600453
:040D3F001DA646C4E3
:040D400015AA40218F
:040D41003BB3500070
:040D42003BB3A0001F
:040D43003124100047
:040D44000205A0EF15
:040D45002E8AE62EDE
:040D46001C05AA8F4F
:040D47001FB2478010
:040D480028AA06606F
:040D49002150000F26
:040D4A000DC61C8135
:040D4B003C8216A12F
:040D4C003105A9972D
:040D4D002924002035
:040D4E002BC602406E
:040D4F001005A9F7EB
:040D50003B280A042E
:040D51003405AA3784
:040D52003B05AA4F64
:040D5300000000009C
:040D540019C201C2FD
:040D550019C201AE10
:040D560038F400006D
:040D570019C206E1D6
:040D580026504C11C4
:040D590026C7B6E310
:040D5A001805AB5776
:040D5B0004C60405C1
:040D5C0032E660001B
:040D5D0038F4000066
:040D5E003DB3F000B1
:040D5F0009861021D0
:040D60003D05AC4061
:040D610001A210617A
:040D62001B8A56256D
:040D63001E05ABC1FD
:040D64001D88E040C6
:040D65001505AB784D
:040D66000CA216E1E4
:040D670032E6600010
:040D680016881000D9
:040D6900323C100008
:040D6A003305A8EFB6
:040D6B000000000084
:040D6C002150000F03
:040D6D0029C7FFEBA8
:040D6E0015A6B70E01
:040D6F0004C603E9CA
:040D70002EC61FEA82
:040D71001B05AE3779
:040D720038F4000051
:040D73001005AE7742
:040D740032E6600003
:040D75003DB3F0009A
:040D76001F05B6F0AF
:040D770039B39001FB
:040D780006A6A0210A
:040D79000B05B9D1DC
:040D7A002AB3E002B6
:040D7B0000A69042FC
:040D7C003782262272
:040D7D000FA6066354
:040D7E000FB310009F
:040D7F000CC8200F6D
:040D80003105B191F7
:040D810009C8200A73
:040D82003105B191F5
:040D83002EC8200551
:040D84003105B191F3
:040D850025C8201F3E
:040D86001E05B59100
:040D870028C8200652
:040D88003105B191EF
:040D89000BC820076C
:040D8A003105B191ED
:040D8B002605B9CFB1
:040D8C003372262C6C
:040D8D00188AC62CCE
:040D8E0029C600086A
:040D8F002BC600056A
:040D90001D05B21774
:040D910003E8000073
:040D92002B82006050
:040D930010B3F107A1
:040D94003105B297DC
:040D950014E66004FC
:040D96003AA64184B4
:040D97000AC8800FF7
:040D98001E05B488F8
:040D990015728084CB
:040D9A001FAA40A5A7
:040D9B00098A16218A
:040D9C003205B51156
:040D9D0013828048F5
:040D9E0005C8801BE9
:040D9F003D05B2104C
:040DA0001AB210A5CE
:040DA10020AA562509
:040DA200063C5000BB
:040DA3001705B1CFB0
:040DA40015727084D0
:040DA5002B8A80E72E
:040DA60015727084CE
:040DA7003505B34F0C
:040DA8001AB210A5C6
:040DA90020AA562501
:040DAA00063C5000B3
:040DAB003505AE2F2D
:040DAC001D05B597D5
:040DAD0003E8000057
:040DAE002B82006034
:040DAF003C05B5F753
:040DB00014E66004E1
:040DB10013B21084E5
:040DB20031AA4624F8
:040DB300343C40008C
:040DB400098A162171
:040DB5003705B581C8
:040DB6003505AE2F22
:040DB70018B350011C
:040DB80032B3A02191
:040DB9001505B7372E
:040DBA0029E8002004
:040DBB0004A6062361
:040DBC002E8AE62E67
:040DBD003905B7B786
:040DBE0014E66004D3
:040DBF0036B2E02543
:040DC0003BB220A57D
:040DC10034A64162B1
:040DC20020AA5045CE
:040DC3001AB210A5AB
:040DC4000AAA5065C2
:040DC5001AB210A5A9
:040DC60020AA5625E4
:040DC700063C500096
:040DC80025A6362303
:040DC9001805AE312A
:040DCA0012AA4625FE
:040DCB000E05B977E1
:040DCC00063C500091
:040DCD003505AE2F0B
:040DCE000000000021
:040DCF001FB2478088
:040DD00028AA0660E7
:040DD1002150000F9E
:040DD2000DC61C81AD
:040DD3003C8216A1A7
:040DD4000005BA97C5
:040DD50029240020AD
:040DD6002BC60240E6
:040DD7002105BAF741
:040DD8003B280A04A6
:040DD9000B05BB3714
:040DDA000405BB4F02
:040DDB000000000014
:040E00001BC20760AA
:040E01002150000F6D
:040E02000BC7FFE13A
:040E030001A6002A1A
:040E04003405C811D8
:040E0500137A00005C
:040E060022A6002BF5
:040E07003405C811D5
:040E08000EC67FE2B1
:040E090007B2C04329
:040E0A003FAA206279
:040E0B000750000B81
:040E0C000CC7FFE927
:040E0D0031C20740A7
:040E0E0013C620E106
:040E0F0002A6002C0B
:040E10003405C811CC
:040E11002AC7CA48DA
:040E12002EB01000EE
:040E13002005C38073
:040E1400137A00004D
:040E15002EC7FFE302
:040E16002EA63003D1
:040E170011C20064A0
:040E18000DC6000102
:040E19001EC6400EA3
:040E1A0006C7CD48F2
:040E1B000705C40FF4
:040E1C00137A000045
:040E1D0021A6002DDD
:040E1E002A05C411CC
:040E1F0008C7C8C870
:040E20001A2C000088
:040E210014C7C680AC
:040E220004C60405F9
:040E2300049056AD34
:040E240011C760E6AC
:040E2500288260A619
:040E2600242400C0C0
:040E270036C761C6A3
:040E2800288260A616
:040E29001AC610A035
:040E2A0000000000C4
:040E2B0000000000C3
:040E2C0000000000C2
:040E2D0000000000C1
:040E2E0000000000C0
:040E2F0000000000BF
:040E30002705C617B5
:040E3100242400C0B5
:040E3200213000006B
:040E33002805C66F59
:040E340009C6000FDC
:040E350000000000B9
:040E36001F389000D1
:040E370000000000B7
:040E38003E38A000A0
:040E390000000000B5
:040E3A000C38B000C0
:040E3B0000000000B3
:040E3C001938C000A1
:040E3D0000000000B1
:040E3E002B38D0007D
:040E3F002B08800FED
:040E40002EC60000BA
:040E41002AC7442157
:040E4200098A1621E2
:040E4300292400203E
:040E44003505C88F19
:040E450000000000A9
:040E46000CE2018039
:040E470026E201A0FE
:040E480005E201A11D
:040E490003B2C0210F
:040E4A0002AA0020D8
:040E4B0002A60040BB
:040E4C000524014038
:040E4D002582A62A2A
:040E4E000AA6A12A25
:040E4F002D8AB62B07
:040E50000C0880000A
:040E51003605D08F03
:040E52000CE201802D
:040E53000CE201802C
:040E5400000000009A
:040E55000000000099
:040E56000000000098
:040E57000000000097
:040E58000000000096
:040E59000000000095
:040E5A000000000094
:040E5B000000000093
:040E5C000000000092
:040E5D000000000091
:040E5E002FE20181FD
:040E5F002FE20181FC
:040E600003B2C021F8
:040E61001AAA1000B9
:040E620002A60040A4
:040E63000524014021
:040E64002582A62A13
:040E65000AA6A12A0E
:040E66002D8AB62BF0
:040E67000000000087
:040E68000C088000F2
:040E69003605D08FEB
:040E6A000CE2018015
:040E6B000CE2018014
:040E6C0002A600409A
:040E6D001BA201C003
:040E6E0003820021DA
:040E6F000A8A462481
:040E70001305CEB1E7
:040E7100000000007D
:040E7200000000007C
:040E7300000000007B
:040E74002B08800FB8
:040E750037241140CD
:040E76002582A62A01
:040E77000AA6A12AFC
:040E78002D8AB62BDE
:040E79003805D090D8
:040E7A000CE2018005
:040E7B000CE2018004
:040E7C0002A600408A
:040E7D0038A201C1D5
:040E7E0011C2006439
:040E7F000A8A462471
:040E80001305CEB1D7
:040E8100000000006D
:040E8200000000006C
:040E83002B08800FA9
:040E84003E38A00054
:040E85000000000069
:040E86000C38B00074
:040E87001A2C000021
:040E88000BC600A1F4
:040E89001305D13745
:040E8A00162410C05A
:040E8B003EC682409D
:040E8C001505D197E0
:040E8D003B280A04F0
:040E8E002004216FAC
:040E8F00000000005F
:040FFE003E04018F1D
:040FFF003E04018F1C
:00000001ff
